:020000040000FA
:04080000B5EF07F059
:1008100003B210EF05F0F2B42BEF05F09EB033EF0A
:1008200005F09EB23BEF05F0F2A81AEF04F0F2B229
:1008300025EF04F0F2A620EF04F0F2B022EF04F06E
:1008400093EF07F0F296F290FF00CD90F2929EA007
:100850002FEF04F00101533F2FEF04F0542BAEC1F2
:10086000B2F1AFC1B3F1B0C1B4F1B1C1B5F1AAC138
:10087000AEF1ABC1AFF1ACC1B0F1ADC1B1F1A6C148
:10088000AAF1A7C1ABF1A8C1ACF1A9C1ADF1A2C158
:10089000A6F1A3C1A7F1A4C1A8F1A5C1A9F19EC168
:1008A000A2F19FC1A3F1A0C1A4F1A1C1A5F19AC178
:1008B0009EF19BC19FF19CC1A0F19DC1A1F196C188
:1008C0009AF197C19BF198C19CF199C19DF1CECF4E
:1008D00096F1CFCF97F153C198F154C199F1CF6AF6
:1008E000CE6A0101536B546B9E90CD800EBC0E8E70
:1008F0000EBA7EEF04F00E8A93EF07F00E8C0EBE58
:10090000BAEF04F096C19AF197C19BF198C19CF19E
:1009100099C19DF19AC19EF19BC19FF19CC1A0F12B
:100920009DC1A1F19EC1A2F19FC1A3F1A0C1A4F1FB
:10093000A1C1A5F1A2C1A6F1A3C1A7F1A4C1A8F1CB
:10094000A5C1A9F1A6C1AAF1A7C1ABF1A8C1ACF19B
:10095000A9C1ADF1AAC1AEF1ABC1AFF1ACC1B0F16B
:10096000ADC1B1F1AEC1B2F1AFC1B3F1B0C1B4F13B
:10097000B1C1B5F101015E6B5F6B606B616B96514C
:100980005E2797515F2398516023995161239A51B3
:100990005E279B515F239C5160239D5161239E5193
:1009A0005E279F515F23A0516023A1516123A25173
:1009B0005E27A3515F23A4516023A5516123A65153
:1009C0005E27A7515F23A8516023A9516123AA5133
:1009D0005E27AB515F23AC516023AD516123AE5113
:1009E0005E27AF515F23B0516023B1516123B251F3
:1009F0005E27B3515F23B4516023B5516123D89072
:100A0000613360335F335E33D890613360335F337B
:100A10005E33D890613360335F335E3393EF07F01A
:100A20000392030103EE00F080517F0BE92604C01E
:100A3000EFFF802B8151805D700BD8A48B8200006A
:100A40008051815D700BD8A48B9281518019D8B4EC
:100A5000079093EF07F0F2940101453F93EF07F001
:100A6000462B93EF07F09E900101533F93EF07F061
:100A7000542B93EF07F09E9204005CA140EF05F029
:100A8000077C07AC5BEF05F0C274C2B455EF05F00C
:100A9000C3CFADF5C4CFAEF50501D890AE33AD33BD
:100AA000D890AE33AD335CEF05F0C3CF55F1C4CF72
:100AB00056F15CEF05F0C28207B4C9EF05F047C1FB
:100AC0004BF148C14CF149C14DF14AC14EF15EC1F3
:100AD00062F15FC163F160C164F161C165F196C10A
:100AE000B6F197C1B7F198C1B8F199C1B9F19AC1FE
:100AF000BAF19BC1BBF19CC1BCF19DC1BDF19EC1CE
:100B0000BEF19FC1BFF1A0C1C0F1A1C1C1F1A2C19D
:100B1000C2F1A3C1C3F1A4C1C4F1A5C1C5F1A6C16D
:100B2000C6F1A7C1C7F1A8C1C8F1A9C1C9F1AAC13D
:100B3000CAF1ABC1CBF1ACC1CCF1ADC1CDF1AEC10D
:100B4000CEF1AFC1CFF1B0C1D0F1B1C1D1F1B2C1DD
:100B5000D2F1B3C1D3F1B4C1D4F1B5C1D5F1ADC5B2
:100B6000AFF5AEC5B0F5AFC5B1F5B0C5B2F5010191
:100B700055515B2756515C23E86A5D230D2EC9EF62
:100B800005F05CC157F15DC158F15B6B5C6B5D6B4F
:100B9000078E0201002F93EF07F03C0E006F00C19B
:100BA0000CF101C10DF102C10EF103C10FF104C13D
:100BB00010F105C111F106C112F107C113F108C10D
:100BC00014F109C115F10AC116F10BC117F134C1B5
:100BD00035F105012951000AD8B492EF06F005015C
:100BE0002951010AD8B41CEF06F005012951020A67
:100BF000D8B45DEF06F005012951030AD8B45DEFC2
:100C000006F005012951040AD8B45DEF06F005018C
:100C10002951050AD8B45DEF06F005012951060AED
:100C2000D8B45DEF06F005012951070AD8B45DEF8D
:100C300006F0296B92EF06F005014D6727EF06F0ED
:100C40004E6727EF06F04F6727EF06F050672BEF50
:100C500006F092EF06F051C500F152C501F153C5FF
:100C600002F154C503F10101010E046F000E056F7E
:100C7000000E066F000E076F8CEC1CF000C151F5E2
:100C800001C152F502C153F503C154F5006750EF9D
:100C900006F0016750EF06F0026750EF06F00367B9
:100CA00092EF06F04DC551F54EC552F54FC553F5BF
:100CB00050C554F50E8892EF06F005012A6763EFE0
:100CC00006F092EF06F00EBE78EF06F00FA07DEF73
:100CD00006F00101476774EF06F0486774EF06F00D
:100CE000496774EF06F04A6778EF06F07DEF06F08B
:100CF00007AE7DEF06F08FEF06F005012B2F92EF88
:100D000006F03C0E2B6F2A2F92EF06F00101000E29
:100D1000626FE00E636FA50E646F010E656F0501D3
:100D20002A6B0E8805015C6B2DB798EF06F05C818D
:100D30000CC100F10DC101F10EC102F10FC103F1AF
:100D400010C104F111C105F112C106F113C107F17F
:100D500014C108F115C109F116C10AF117C10BF14F
:100D600035C134F100C10CF101C10DF102C10EF128
:100D700003C10FF104C110F105C111F106C112F157
:100D800007C113F108C114F109C115F10AC116F127
:100D90000BC117F134C135F101018A67D7EF06F0B5
:100DA0008B67D7EF06F08C67D7EF06F08D67DBEF28
:100DB00006F00BEF07F08EC100F18FC101F190C179
:100DC00002F191C103F10101010E046F000E056FE4
:100DD000000E066F000E076F8CEC1CF000C18EF148
:100DE00001C18FF102C190F103C191F1006700EFE1
:100DF00007F0016700EF07F0026700EF07F00367F5
:100E00000BEF07F08AC18EF18BC18FF18CC190F18D
:100E10008DC191F10E80D57ED5BE69D0D6CF47F178
:100E2000D7CF48F145C149F1E86AE8CF4AF10F90C0
:100E300047C100F148C101F149C102F14AC103F1C2
:100E400001010A0E046F000E056F000E066F000E02
:100E5000076F8CEC1CF000AF0F80010154A73DEF31
:100E600007F00E9A0E9C0E9E0101000E5E6F600E42
:100E70005F6F3D0E606F080E616F010147BF4DEF60
:100E800007F048674DEF07F049674DEF07F04A67F5
:100E90004DEF07F0F28872EF07F0F2985E6B5F6B30
:100EA000606B616B966B976B986B996B9A6B9B6B96
:100EB0009C6B9D6B9E6B9F6BA06BA16BA26BA36BDE
:100EC000A46BA56BA66BA76BA86BA96BAA6BAB6B8E
:100ED000AC6BAD6BAE6BAF6BB06BB16BB26BB36B3E
:100EE000B46BB56BD76AD66A0101456B466B0CC112
:100EF00000F10DC101F10EC102F10FC103F110C1EA
:100F000004F111C105F112C106F113C107F114C1B9
:100F100008F115C109F116C10AF117C10BF135C16C
:100F200034F193EF07F002C0E0FF005001C0D8FF9A
:100F30001000A6B299EF07F00CC0A9FF0BC0A8FFE4
:100F4000A69EA69CA684F29E550EA76EAA0EA76E1C
:100F5000A682F28EA694A6B2ABEF07F01200A96E9D
:100F6000A69EA69CA680A8501200076A0E6A0F6A69
:100F70000F010D0EC16E860EC06E030EC26E0F0104
:100F8000280E896E130E926E080E8A6EF30E936E03
:100F90008B6A900E946EF18EF19E0D6A01015B6B6F
:100FA0005C6B5D6B576B586BF29A0101476B486B3A
:100FB000496B4A6B4B6B4C6B4D6B4E6B4F6B506B75
:100FC000516B526B456B466BD76AD66A0F01280E80
:100FD000D56EF28A9D90B00ECD6E01015E6B5F6B97
:100FE000606B616B626B636B646B656B666B676B8D
:100FF000686B696B536B546BCF6ACE6A0E9A0E9C0A
:101000000E9E9D80760ECA6E9D8202013C0E006F80
:10101000CC6A160EAFEC07F0E8CF00F1170EAFEC7C
:1010200007F0E8CF01F1180EAFEC07F0E8CF02F1BE
:10103000190EAFEC07F0E8CF03F1010103AF3BEF6E
:1010400008F083EC1DF0160E0C6E00C10BF099EC4D
:1010500007F0170E0C6E01C10BF099EC07F0180E9B
:101060000C6E02C10BF099EC07F0190E0C6E03C167
:101070000BF099EC07F000C18AF101C18BF102C1BC
:101080008CF103C18DF100C18EF101C18FF102C15C
:1010900090F103C191F11A0EAFEC07F0E8CF00F127
:1010A0001B0EAFEC07F0E8CF01F11C0EAFEC07F020
:1010B000E8CF02F11D0EAFEC07F0E8CF03F101011C
:1010C00003AF91EF08F083EC1DF01A0E0C6E00C117
:1010D0000BF099EC07F01B0E0C6E01C10BF099ECB4
:1010E00007F01C0E0C6E02C10BF099EC07F01D0E00
:1010F0000C6E03C10BF099EC07F01A0EAFEC07F081
:10110000E8CF00F11B0EAFEC07F0E8CF01F11C0EA9
:10111000AFEC07F0E8CF02F11D0EAFEC07F0E8CF1F
:1011200003F100C192F101C193F102C194F103C135
:1011300095F1240EAC6E900EAB6E240EAC6E080EC4
:10114000B86E000EB06E1F0EAF6E0401806B816B27
:101150000F01900EAB6E0F019D8A0301806B816BB6
:10116000A26B8B92D1EC20F0200EAFEC07F0E8CF11
:1011700029F505012951FF0AD8A4C6EF08F0296B0B
:10118000200E0C6E29C50BF099EC07F00501010E3D
:101190002A6F3C0E2B6F250EAFEC07F0E8CF00F165
:1011A000260EAFEC07F0E8CF01F1270EAFEC07F009
:1011B000E8CF02F1280EAFEC07F0E8CF03F1010110
:1011C00003AFFDEF08F083EC1DF0250E0C6E00C19F
:1011D0000BF099EC07F0260E0C6E01C10BF099ECA8
:1011E00007F0270E0C6E02C10BF099EC07F0280EE9
:1011F0000C6E03C10BF099EC07F000C14DF501C175
:101200004EF502C14FF503C150F500C151F501C1C2
:1012100052F502C153F503C154F5290EAFEC07F0A6
:10122000E8CF55F505015651555DD8A055C556F581
:1012300005012951020A0EE181B82AEF09F00501E2
:10124000562F27EF09F055C556F52AEF09F081BA58
:10125000F0EF23F0210EAFEC07F0E8CF00F1220E03
:10126000AFEC07F0E8CF01F1230EAFEC07F0E8CFC9
:1012700002F1240EAFEC07F0E8CF03F1010103AF58
:1012800070EF09F083EC1DF0210E0C6E00C10BF025
:1012900099EC07F0220E0C6E01C10BF099EC07F0EF
:1012A000230E0C6E02C10BF099EC07F0240E0C6EAD
:1012B00003C10BF099EC07F0210EAFEC07F0E8CF7B
:1012C00000F1220EAFEC07F0E8CF01F1230EAFECF6
:1012D00007F0E8CF02F1240EAFEC07F0E8CF03F1FE
:1012E00000C157F501C158F502C159F503C15AF5BE
:1012F00008EC20F0CAEC1EF0F0EC1DF005012951BD
:10130000030A12E005012951040A1DE005012951D3
:10131000050A24E005012951060A32E00501295198
:10132000070A38E0D3EF09F0A6C500F101010F0E5E
:10133000001701010051000A36E001010051050AC1
:1013400032E0D0EF09F0A6C500F101010F0E001741
:1013500001010051000A27E0D0EF09F00501A65174
:10136000000A21E00501A651150A1DE00501A6515C
:10137000300A19E00501A651450A15E0D0EF09F041
:101380000501A651000A0FE00501A651300A0BE045
:10139000D0EF09F00501A651000A05E0D0EF09F0F1
:1013A00081BAF0EF23F007900001F28EF28C07B0C3
:1013B00003EF1AF00EB0E4EF14F00EB8D6EF0EF013
:1013C0000301805181197F0BD8B403EF1AF013EE9B
:1013D00000F081517F0BE126812BE7CFE8FFE00B86
:1013E000D8B403EF1AF023EE82F0A2511F0BD926D6
:1013F000E7CFDFFFA22BDF50780AD8A403EF1AF063
:1014000007808EC100F18FC101F190C102F191C13D
:1014100003F10101040E046F000E056F000E066F4C
:10142000000E076F8CEC1CF000AF20EF0AF00101FA
:10143000030E8E6F000E8F6F000E906F000E916F77
:1014400003018251720AD8B4E4EF14F08251520AB7
:10145000D8B4E4EF14F08251750AD8B4E4EF14F074
:101460008251630AD8B4BFEF16F08251690AD8B42A
:101470009FEF11F082517A0AD8B4B2EF12F0825184
:10148000490AD8B43EEF11F08251500AD8B45CEF4B
:1014900010F08251700AD8B49FEF10F08251540AB4
:1014A000D8B4CAEF10F08251740AD8B410EF11F01A
:1014B0008251730AD8B414EF14F08251530AD8B48D
:1014C00079EF14F082514C0AD8B47CEF0AF0F4EFB3
:1014D00016F0040114EE00F080517F0BE12682C467
:1014E000E7FF802B12000D0E826F69EC0AF00A0EE6
:1014F000826F69EC0AF0120003018351300AD8B4FC
:101500002BEF0DF003018351310AD8B4B1EF0DF088
:1015100003018351320AD8B401EF0EF00301835165
:10152000330AD8B405EF0EF003018351340AD8B45E
:1015300013EF0EF003018351350AD8B4DBEF0EF040
:10154000030183514D0AD8B4A4EF0BF0030183517A
:101550006D0AD8B4BEEF0BF003018351490AD8B429
:10156000DBEF0FF003018351500AD8B40DEF0FF0F9
:1015700003018351540AD8B486EF0FF0030183515D
:10158000630AD8B4DEEF0BF003018351430AD8B4E9
:10159000D6EF0CF003018351730AD8B4DCEF0BF0E3
:1015A00003018351610AD8B4F1EF0AF003018351BA
:1015B000650AD8B479EF0DF003018351450AD8B418
:1015C00087EF0DF003018351620AD8B495EF0DF057
:1015D00003018351420AD8B4A3EF0DF0D8A4F4EF6D
:1015E00016F004014C0E826F69EC0AF00401610EE2
:1015F000826F69EC0AF0CAEC1EF004012C0E826FB7
:1016000069EC0AF083EC1DF0A5C500F1010126ECA0
:101610001DF031C182F40401300E822769EC0AF01A
:1016200032C182F40401300E822769EC0AF033C122
:1016300082F40401300E822769EC0AF004012C0EBA
:10164000826F69EC0AF083EC1DF0A6C500F1010180
:1016500026EC1DF031C182F40401300E822769ECC2
:101660000AF032C182F40401300E822769EC0AF0DC
:1016700033C182F40401300E822769EC0AF00401C0
:101680002C0E826F69EC0AF083EC1DF0A7C500F107
:10169000010126EC1DF031C182F40401300E8227D5
:1016A00069EC0AF032C182F40401300E822769EC41
:1016B0000AF033C182F40401300E822769EC0AF08B
:1016C00004012C0E826F69EC0AF083EC1DF0A8C5B2
:1016D00000F1010126EC1DF031C182F40401300E4D
:1016E000822769EC0AF032C182F40401300E8227AD
:1016F00069EC0AF033C182F40401300E822769ECF0
:101700000AF004012C0E826F69EC0AF083EC1DF0E4
:10171000ADC500F1010126EC1DF031C182F40401D8
:10172000300E822769EC0AF032C182F40401300ED7
:10173000822769EC0AF033C182F40401300E82275B
:1017400069EC0AF009EF0FF0C4EC1DF084C333F12B
:10175000D1EC1DF048EC1DF0200E0C6E00C10BF01A
:1017600099EC07F000C129F505012951000A06E0AE
:1017700005012951010A02E070EC1FF004014C0E32
:10178000826F69EC0AF004014D0E826F69EC0AF079
:1017900004012C0E826F69EC0AF083EC1DF029C560
:1017A00000F126EC1DF033C182F40401300E8227D3
:1017B00069EC0AF009EF0FF0F0EF23F004014C0E92
:1017C000826F69EC0AF00401630E826F69EC0AF023
:1017D000F0EC1DF004012C0E826F69EC0AF0F3ECC2
:1017E0000BF009EF0FF083EC1DF0ABC500F1010128
:1017F000003B0F0E001726EC1DF033C182F40401EC
:10180000300E822769EC0AF0ABC500F101010F0E22
:101810000101001726EC1DF033C182F40401300EE3
:10182000822769EC0AF004012D0E826F69EC0AF040
:10183000AAC500F10101003B0F0E001726EC1DF0B8
:1018400033C182F40401300E822769EC0AF0AAC584
:1018500000F101010F0E0101001726EC1DF033C14C
:1018600082F40401300E822769EC0AF004012D0E87
:10187000826F69EC0AF0A9C500F10101003B0F0E6F
:10188000001726EC1DF033C182F40401300E8227CC
:1018900069EC0AF0A9C500F101010F0E0101001762
:1018A00026EC1DF033C182F40401300E822769EC6E
:1018B0000AF00401200E826F69EC0AF0A8C500F15D
:1018C0000F0E0101001726EC1DF033C182F4040154
:1018D000300E822769EC0AF00401200E826F69EC59
:1018E0000AF0A7C500F101010101003B0F0E00172E
:1018F00026EC1DF033C182F40401300E822769EC1E
:101900000AF0A7C500F101010F0E0101001726EC36
:101910001DF033C182F40401300E822769EC0AF015
:1019200004013A0E826F69EC0AF0A6C500F10101CC
:10193000003B0F0E001726EC1DF033C182F40401AA
:10194000300E822769EC0AF0A6C500F101010F0EE6
:101950000101001726EC1DF033C182F40401300EA2
:10196000822769EC0AF004013A0E826F69EC0AF0F2
:10197000A5C500F10101003B0F0E001726EC1DF07C
:1019800033C182F40401300E822769EC0AF0A5C548
:1019900000F101010F0E001726EC1DF033C182F497
:1019A0000401300E822769EC0AF0120084C3E8FFBC
:1019B0000F0BE83AE8CFABF585C3E8FF0F0B050145
:1019C000AB1387C3E8FF0F0BE83AE8CFAAF588C34B
:1019D000E8FF0F0B0501AA138AC3E8FF0F0BE83AD3
:1019E000E8CFA9F58BC3E8FF0F0B0501A9138DC341
:1019F000E8FF0F0BE8CFA8F58FC3E8FF0F0BE83A1D
:101A0000E8CFA7F590C3E8FF0F0B0501A71392C31A
:101A1000E8FF0F0BE83AE8CFA6F593C3E8FF0F0BFA
:101A20000501A61395C3E8FF0F0BE83AE8CFA5F52B
:101A300096C3E8FF0F0B0501A5134FEC1EF0040140
:101A40004C0E826F69EC0AF00401430E826F69EC60
:101A50000AF0E8EF0BF0B1EC23F083EC1DF02DC59C
:101A600000F126EC1DF004014C0E826F69EC0AF0C7
:101A70000401300E826F69EC0AF004012C0E826FB3
:101A800069EC0AF031C182F40401300E822769EC5E
:101A90000AF032C182F40401300E822769EC0AF0A8
:101AA00033C182F40401300E822769EC0AF004018C
:101AB0002C0E826F69EC0AF083EC1DF02EC500F14C
:101AC00026EC1DF031C182F40401300E822769EC4E
:101AD0000AF032C182F40401300E822769EC0AF068
:101AE00033C182F40401300E822769EC0AF009EF59
:101AF0000FF004014C0E826F69EC0AF00401650ED0
:101B0000826F69EC0AF059EC20F009EF0FF0040144
:101B10004C0E826F69EC0AF00401450E826F69EC8D
:101B20000AF076EC20F009EF0FF004014C0E826F02
:101B300069EC0AF00401620E826F69EC0AF0B0EC05
:101B400020F009EF0FF004014C0E826F69EC0AF0EF
:101B50000401420E826F69EC0AF093EC20F009EF69
:101B60000FF004014C0E826F69EC0AF00401310E93
:101B7000826F69EC0AF004012C0E826F69EC0AF0A6
:101B800025C500F126C501F127C502F128C503F1DD
:101B90000101100E046F000E056F000E066F000E9F
:101BA000076FBAEC1CF026EC1DF02EC182F4040184
:101BB000300E822769EC0AF02FC182F40401300E46
:101BC000822769EC0AF030C182F40401300E8227CA
:101BD00069EC0AF031C182F40401300E822769EC0D
:101BE0000AF032C182F40401300E822769EC0AF057
:101BF00033C182F40401300E822769EC0AF009EF48
:101C00000FF01BEC21F0F4EF16F004014C0E826F84
:101C100069EC0AF00401330E826F69EC0AF051ECB2
:101C200021F0BBEF0DF004014C0E826F69EC0AF05D
:101C30000401340E826F69EC0AF004012C0E826FED
:101C400069EC0AF0C4EC1DF084C32AF185C32BF1C2
:101C500086C32CF187C32DF188C32EF189C32FF1E0
:101C60008AC330F18BC331F18CC332F18DC333F1B0
:101C70000101296BD1EC1DF048EC1DF0100E046F32
:101C8000000E056F000E066F000E076F9BEC1CF038
:101C900000C121F501C122F502C123F503C124F5DC
:101CA00064EC23F02EC5A5F52FC5A6F530C5A7F524
:101CB00031C5A8F532C5A9F533C5AAF534C5ABF5CC
:101CC000F3EC0BF004012C0E826F69EC0AF035C5C1
:101CD00000F136C501F137C502F138C503F1010144
:101CE000000E046F000E056F010E066F000E076FE9
:101CF000BAEC1CF026EC1DF0296781EF0EF086EFA0
:101D00000EF004012D0E826F69EC0AF030C182F4EE
:101D10000401300E822769EC0AF031C182F404011B
:101D2000300E822769EC0AF004012E0E826F69ECF6
:101D30000AF032C182F40401300E822769EC0AF005
:101D400033C182F40401300E822769EC0AF00401E9
:101D50002C0E826F69EC0AF083EC1DF039C500F19E
:101D60003AC501F11EEC18F004012C0E826F69ECEB
:101D70000AF083EC1DF03BC500F126EC1DF031C1EB
:101D800082F40401300E822769EC0AF032C182F439
:101D90000401300E822769EC0AF033C182F4040199
:101DA000300E822769EC0AF009EF0FF00E9851EC23
:101DB00021F009EF0FF004014C0E826F69EC0AF07C
:101DC0000401350E826F69EC0AF004012C0E826F5B
:101DD00069EC0AF083EC1DF00784AFC500F10794AD
:101DE00026EC1DF031C182F40401300E822769EC2B
:101DF0000AF032C182F40401300E822769EC0AF045
:101E000033C182F40401300E822769EC0AF009EF35
:101E10000FF073EC0AF0F4EF16F004014C0E826F31
:101E200069EC0AF00401500E826F69EC0AF00401BB
:101E30002C0E826F69EC0AF085C32AF186C32BF160
:101E400087C32CF188C32DF189C32EF18AC32FF1EA
:101E50008BC330F18CC331F18DC332F18EC333F1BA
:101E60000101D1EC1DF048EC1DF003018451530A2F
:101E70000DE0030184514D0A38E00401780E826FB1
:101E800069EC0AF073EC0AF0F4EF16F00401530E5B
:101E9000826F69EC0AF0250E0C6E00C10BF099EC14
:101EA00007F0260E0C6E01C10BF099EC07F0270E1F
:101EB0000C6E02C10BF099EC07F0280E0C6E03C1FA
:101EC0000BF099EC07F000C14DF501C14EF502C1D0
:101ED0004FF503C150F500C151F501C152F502C1E2
:101EE00053F503C154F5EAEF0FF004014D0E826F74
:101EF00069EC0AF0290E0C6E00C10BF099EC07F0AA
:101F000000C155F500C156F5EAEF0FF004014C0E83
:101F1000826F69EC0AF00401540E826F69EC0AF0DA
:101F200004012C0E826F69EC0AF084C32AF185C388
:101F30002BF186C32CF187C32DF188C32EF189C301
:101F40002FF18AC330F18BC331F18DC332F18EC3CF
:101F500033F10101D1EC1DF048EC1DF00101000E40
:101F6000046F000E056F010E066F000E076F9BECED
:101F70001CF0210E0C6E00C10BF099EC07F0220E44
:101F80000C6E01C10BF099EC07F0230E0C6E02C130
:101F90000BF099EC07F0240E0C6E03C10BF099ECDA
:101FA00007F000C157F501C158F502C159F503C149
:101FB0005AF5EAEF0FF004014C0E826F69EC0AF05B
:101FC0000401490E826F69EC0AF004012C0E826F45
:101FD00069EC0AF0250EAFEC07F0E8CF00F1260E11
:101FE000AFEC07F0E8CF01F1270EAFEC07F0E8CF38
:101FF00002F1280EAFEC07F0E8CF03F126EC1DF05C
:1020000031EC1BF00401730E826F69EC0AF00401DD
:102010002C0E826F69EC0AF083EC1DF0290EAFECF8
:1020200007F0E8CF00F126EC1DF031EC1BF00401C5
:10203000730E826F69EC0AF004012C0E826F69EC5A
:102040000AF051C500F152C501F153C502F154C562
:1020500003F126EC1DF031EC1BF00401730E826FCE
:1020600069EC0AF004012C0E826F69EC0AF083EC33
:102070001DF056C500F126EC1DF031EC1BF00401FB
:102080006D0E826F69EC0AF004012C0E826F69EC10
:102090000AF057C500F158C501F159C502F15AC5FA
:1020A00003F10FEC17F004012C0E826F69EC0AF0BB
:1020B00073EC0AF0F4EF16F083C32AF184C32BF11A
:1020C00085C32CF186C32DF187C32EF188C32FF170
:1020D00089C330F18AC331F18BC332F18CC333F140
:1020E0000101D1EC1DF048EC1DF0160E0C6E00C184
:1020F0000BF099EC07F0170E0C6E01C10BF099EC88
:1021000007F0180E0C6E02C10BF099EC07F0190ED7
:102110000C6E03C10BF099EC07F000C18AF101C10C
:102120008BF102C18CF103C18DF100C18EF101C1AF
:102130008FF102C190F103C191F13EEF11F083C321
:102140002AF184C32BF185C32CF186C32DF187C3FB
:102150002EF188C32FF189C330F18AC331F18BC3CB
:1021600032F18CC333F10101D1EC1DF048EC1DF0CC
:1021700000C18AF101C18BF102C18CF103C18DF163
:1021800000C18EF101C18FF102C190F103C191F143
:102190003EEF11F083C32AF184C32BF185C32CF1E8
:1021A00086C32DF187C32EF188C32FF189C330F187
:1021B0008AC331F18CC332F18DC333F10101D1EC0B
:1021C0001DF048EC1DF00101000E046F000E056FBC
:1021D000010E066F000E076F9BEC1CF01A0E0C6EC2
:1021E00000C10BF099EC07F01B0E0C6E01C10BF057
:1021F00099EC07F01C0E0C6E02C10BF099EC07F085
:102200001D0E0C6E03C10BF099EC07F000C192F1AA
:1022100001C193F102C194F103C195F13EEF11F0B8
:1022200083C32AF184C32BF185C32CF186C32DF11E
:1022300087C32EF188C32FF189C330F18AC331F1EE
:102240008CC332F18DC333F10101D1EC1DF048ECA8
:102250001DF00101000E046F000E056F010E066FE8
:10226000000E076F9BEC1CF000C192F101C193F1CD
:1022700002C194F103C195F13EEF11F0160EAFECDF
:1022800007F0E8CF00F1170EAFEC07F0E8CF01F14F
:10229000180EAFEC07F0E8CF02F1190EAFEC07F023
:1022A000E8CF03F126EC1DF031EC1BF00401730EB6
:1022B000826F69EC0AF004012C0E826F69EC0AF05F
:1022C0008AC100F18BC101F18CC102F18DC103F112
:1022D00026EC1DF031EC1BF00401730E826F69ECEB
:1022E0000AF004012C0E826F69EC0AF01A0EAFECB2
:1022F00007F0E8CF00F11B0EAFEC07F0E8CF01F1DB
:102300001C0EAFEC07F0E8CF02F11D0EAFEC07F0AA
:10231000E8CF03F10FEC17F004012C0E826F69EC8B
:102320000AF092C100F193C101F194C102F195C18B
:1023300003F10FEC17F073EC0AF0F4EF16F0040160
:10234000690E826F69EC0AF004012C0E826F69EC51
:102350000AF00101040E006F000E016F000E026F03
:10236000000E036F26EC1DF02CC182F40401300E28
:10237000822769EC0AF02DC182F40401300E822715
:1023800069EC0AF02EC182F40401300E822769EC58
:102390000AF02FC182F40401300E822769EC0AF0A2
:1023A00030C182F40401300E822769EC0AF031C199
:1023B00082F40401300E822769EC0AF032C182F403
:1023C0000401300E822769EC0AF033C182F4040163
:1023D000300E822769EC0AF004012C0E826F69EC42
:1023E0000AF00101060E006F000E016F000E026F71
:1023F000000E036F26EC1DF02CC182F40401300E98
:10240000822769EC0AF02DC182F40401300E822784
:1024100069EC0AF02EC182F40401300E822769ECC7
:102420000AF02FC182F40401300E822769EC0AF011
:1024300030C182F40401300E822769EC0AF031C108
:1024400082F40401300E822769EC0AF032C182F472
:102450000401300E822769EC0AF033C182F40401D2
:10246000300E822769EC0AF004012C0E826F69ECB1
:102470000AF00101190E006F000E016F000E026FCD
:10248000000E036F26EC1DF02CC182F40401300E07
:10249000822769EC0AF02DC182F40401300E8227F4
:1024A00069EC0AF02EC182F40401300E822769EC37
:1024B0000AF02FC182F40401300E822769EC0AF081
:1024C00030C182F40401300E822769EC0AF031C178
:1024D00082F40401300E822769EC0AF032C182F4E2
:1024E0000401300E822769EC0AF033C182F4040142
:1024F000300E822769EC0AF004012C0E826F69EC21
:102500000AF0200EF86EF76AF66A04010900F5CFAA
:1025100082F469EC0AF00900F5CF82F469EC0AF064
:102520000900F5CF82F469EC0AF00900F5CF82F4D6
:1025300069EC0AF00900F5CF82F469EC0AF00900B1
:10254000F5CF82F469EC0AF00900F5CF82F469EC6A
:102550000AF00900F5CF82F469EC0AF073EC0AF096
:10256000F4EF16F08351630AD8A4F4EF16F0845107
:10257000610AD8A4F4EF16F085516C0AD8A4F4EFE0
:1025800016F08651410A42E08651440A1BE086510A
:10259000420AD8B419EF13F08651350AD8B47EEF49
:1025A00018F08651360AD8B4D3EF18F08651370A9E
:1025B000D8B43CEF19F08651380AD8B49AEF19F024
:1025C000F4EF16F00798079A04017A0E826F69EC0F
:1025D0000AF00401780E826F69EC0AF00401640EBF
:1025E000826F69EC0AF081A8FDEF12F00401550E2C
:1025F000826F69EC0AF002EF13F004014C0E826F57
:1026000069EC0AF073EC0AF0F4EF16F00788079A09
:1026100004017A0E826F69EC0AF00401410E826FA8
:1026200069EC0AF00401610E826F69EC0AF0F3EFC5
:1026300012F00798078A04017A0E826F69EC0AF09B
:102640000401420E826F69EC0AF00401610E826F90
:1026500069EC0AF0F3EF12F00101666737EF13F04F
:10266000676737EF13F0686737EF13F069674FEF6D
:1026700013F04F6743EF13F0506743EF13F05167C8
:1026800043EF13F052674FEF13F00101000E006F9C
:10269000000E016F000E026F000E036F12000101A9
:1026A000620E046F010E056F000E066F000E076FBD
:1026B00066C100F167C101F168C102F169C103F1AE
:1026C0008CEC1CF003BFD3EF13F00101000E046F7C
:1026D000A80E056F550E066F020E076F66C100F15A
:1026E00067C101F168C102F169C103F166C186F1F8
:1026F00067C187F168C188F169C189F18CEC1CF070
:1027000003BF8CEF13F00101000E866FA80E876FD8
:10271000550E886F020E896F0E0EAFEC07F0E8CFF2
:1027200018F10F0EAFEC07F0E8CF19F1100EAFEC77
:1027300007F0E8CF1AF1110EAFEC07F0E8CF1BF16C
:10274000D5EC1BF086C104F187C105F188C106F103
:1027500089C107F18CEC1CF0078299EC1BF0D5ECD9
:102760001BF0079299EC1BF086C100F187C101F1C3
:1027700088C102F189C103F1079299EC1BF0CC0EDC
:10278000046FE00E056F870E066F050E076F8CEC69
:102790001CF000C118F101C119F102C11AF103C105
:1027A0001BF10BEF14F00101800E006F1A0E016F88
:1027B000060E026F000E036F4FC104F150C105F108
:1027C00051C106F152C107F18CEC1CF003AFECEFE4
:1027D00013F083EC1DF012000E0EAFEC07F0E8CF03
:1027E00018F10F0EAFEC07F0E8CF19F1100EAFECB7
:1027F00007F0E8CF1AF1110EAFEC07F0E8CF1BF1AC
:102800004FC100F150C101F151C102F152C103F1B8
:10281000078299EC1BF018C100F119C101F11AC12E
:1028200002F11BC103F112000401730E826F69EC07
:102830000AF004012C0E826F69EC0AF0078462C171
:1028400066F163C167F164C168F165C169F14BC1AB
:102850004FF14CC150F14DC151F14EC152F157C130
:1028600059F158C15AF107943AEC14F073EC0AF09C
:10287000F4EF16F066C100F167C101F168C102F121
:1028800069C103F1010126EC1DF031EC1BF00401DC
:10289000630E826F69EC0AF004012C0E826F69EC02
:1028A0000AF04FC100F150C101F151C102F152C112
:1028B00003F1010126EC1DF031EC1BF00401660E62
:1028C000826F69EC0AF004012C0E826F69EC0AF049
:1028D00083EC1DF059C100F15AC101F1010126EC50
:1028E0001DF031EC1BF00401740E826F69EC0AF0EC
:1028F00012000F820401530E826F69EC0AF004018A
:102900002C0E826F69EC0AF083C32AF184C32BF189
:1029100085C32CF186C32DF187C32EF188C32FF117
:1029200089C330F18AC331F18BC332F18CC333F1E7
:102930000101D1EC1DF048EC1DF000C166F101C1B0
:1029400067F102C168F103C169F18EC32AF18FC337
:102950002BF190C32CF191C32DF192C32EF193C3AF
:102960002FF194C330F195C331F196C332F197C37F
:1029700033F10101D1EC1DF048EC1DF000C14FF125
:1029800001C150F102C151F103C152F1C4EC1DF07B
:1029900099C32FF19AC330F19BC331F19CC332F13B
:1029A0009DC333F10101D1EC1DF048EC1DF000C1D5
:1029B00059F101C15AF13AEC14F004012C0E826F66
:1029C00069EC0AF0EBEF14F08251520A03E10E8237
:1029D000EBEF14F00E928251750A03E10F84F2EFCF
:1029E00014F00F948251550A03E10F86F9EF14F0A9
:1029F0000F9607840FB256EF15F00FA442EF15F0B3
:102A0000B6C166F1B7C167F1B8C168F1B9C169F182
:102A1000BAC16AF1BBC16BF1BCC16CF1BDC16DF152
:102A2000BEC16EF1BFC16FF1C0C170F1C1C171F122
:102A3000C2C172F1C3C173F1C4C174F1C5C175F1F2
:102A4000C6C176F1C7C177F1C8C178F1C9C179F1C2
:102A5000CAC17AF1CBC17BF1CCC17CF1CDC17DF192
:102A6000CEC17EF1CFC17FF1D0C180F1D1C181F162
:102A7000D2C182F1D3C183F1D4C184F1D5C185F132
:102A80004AEF15F062C166F163C167F164C168F194
:102A900065C169F14BC14FF14CC150F14DC151F1CC
:102AA0004EC152F157C159F158C15AF107940EA0C5
:102AB00078EF15F00101926765EF15F0936765EF08
:102AC00015F0946765EF15F0956769EF15F078EFED
:102AD00015F02CEC13F092C104F193C105F194C1EF
:102AE00006F195C107F18CEC1CF003BFBCEF16F0AA
:102AF0002CEC13F00101000E046F000E056F010EA7
:102B0000066F000E076FBAEC1CF00FA48FEF15F0E4
:102B10000401750E826F69EC0AF094EF15F0040160
:102B2000720E826F69EC0AF004012C0E826F69EC60
:102B30000AF026EC1DF02967A3EF15F00401200E22
:102B4000826FA6EF15F004012D0E826F69EC0AF07A
:102B500030C182F40401300E822769EC0AF031C1E1
:102B600082F40401300E822769EC0AF004012E0E73
:102B7000826F69EC0AF032C182F40401300E8227C0
:102B800069EC0AF033C182F40401300E822769EC4B
:102B90000AF004016D0E826F69EC0AF004012C0E3C
:102BA000826F69EC0AF04FC100F150C101F151C1CF
:102BB00002F152C103F1010126EC1DF031EC1BF0D2
:102BC0000401480E826F69EC0AF004017A0E826FEC
:102BD00069EC0AF004012C0E826F69EC0AF066C100
:102BE00000F167C101F168C102F169C103F101019E
:102BF00026EC1DF031EC1BF00401630E826F69ECD2
:102C00000AF004012C0E826F69EC0AF066C100F133
:102C100067C101F168C102F169C103F101010A0E46
:102C2000046F000E056F000E066F000E076F9BEC21
:102C30001CF0000E046F120E056F000E066F000EE2
:102C4000076FBAEC1CF026EC1DF02AC182F40401D7
:102C5000300E822769EC0AF02BC182F40401300E99
:102C6000822769EC0AF02CC182F40401300E82271D
:102C700069EC0AF02DC182F40401300E822769EC60
:102C80000AF02EC182F40401300E822769EC0AF0AA
:102C90002FC182F40401300E822769EC0AF030C1A2
:102CA00082F40401300E822769EC0AF004012E0E32
:102CB000826F69EC0AF031C182F40401300E822780
:102CC00069EC0AF032C182F40401300E822769EC0B
:102CD0000AF033C182F40401300E822769EC0AF055
:102CE0000401730E826F69EC0AF004012C0E826FEE
:102CF00069EC0AF083EC1DF059C100F15AC101F1F1
:102D00001EEC18F00EB288EF16F00EA0BAEF16F017
:102D100004012C0E826F69EC0AF0200EF86EF76A3F
:102D2000F66A04010900F5CF82F469EC0AF00900A3
:102D3000F5CF82F469EC0AF00900F5CF82F469EC72
:102D40000AF00900F5CF82F469EC0AF00900F5CF2A
:102D500082F469EC0AF00900F5CF82F469EC0AF01C
:102D60000900F5CF82F469EC0AF00900F5CF82F48E
:102D700069EC0AF073EC0AF00E90F4EF16F004011F
:102D8000630E826F69EC0AF004012C0E826F69EC0D
:102D90000AF0FAEC16F004012C0E826F69EC0AF0CE
:102DA0006DEC17F004012C0E826F69EC0AF0E9EC6F
:102DB00017F004012C0E826F69EC0AF00101F80E85
:102DC000006FCD0E016F660E026F030E036F0FECE6
:102DD00017F004012C0E826F69EC0AF0FFEC17F07B
:102DE00073EC0AF0F4EF16F00301A26B07900F9258
:102DF00003EF1AF0D8900E0EAFEC07F0E8CF00F119
:102E00000F0EAFEC07F0E8CF01F1100EAFEC07F0BA
:102E1000E8CF02F1110EAFEC07F0E8CF03F10101AA
:102E2000000E046F000E056F010E066F000E076F97
:102E3000BAEC1CF026EC1DF02AC182F40401300E1D
:102E4000822769EC0AF02BC182F40401300E82273C
:102E500069EC0AF02CC182F40401300E822769EC7F
:102E60000AF02DC182F40401300E822769EC0AF0C9
:102E70002EC182F40401300E822769EC0AF02FC1C2
:102E800082F40401300E822769EC0AF030C182F42A
:102E90000401300E822769EC0AF031C182F404018A
:102EA000300E822769EC0AF004012E0E826F69EC65
:102EB0000AF032C182F40401300E822769EC0AF074
:102EC00033C182F40401300E822769EC0AF0040158
:102ED0006D0E826F69EC0AF01200120EAFEC07F073
:102EE000E8CF00F1130EAFEC07F0E8CF01F1140EBC
:102EF000AFEC07F0E8CF02F1150EAFEC07F0E8CF2A
:102F000003F101010A0E046F000E056F000E066F3B
:102F1000000E076F9BEC1CF0000E046F120E056F85
:102F2000000E066F000E076FBAEC1CF026EC1DF0C9
:102F30002AC182F40401300E822769EC0AF02BC109
:102F400082F40401300E822769EC0AF02CC182F46D
:102F50000401300E822769EC0AF02DC182F40401CD
:102F6000300E822769EC0AF02EC182F40401300E83
:102F7000822769EC0AF02FC182F40401300E822707
:102F800069EC0AF030C182F40401300E822769EC4A
:102F90000AF004012E0E826F69EC0AF031C182F44E
:102FA0000401300E822769EC0AF032C182F4040178
:102FB000300E822769EC0AF033C182F40401300E2E
:102FC000822769EC0AF00401730E826F69EC0AF043
:102FD00012000A0EAFEC07F0E8CF00F10B0EAFECD9
:102FE00007F0E8CF01F10C0EAFEC07F0E8CF02F1EB
:102FF0000D0EAFEC07F0E8CF03F11EEF18F0060E50
:10300000AFEC07F0E8CF00F1070EAFEC07F0E8CF28
:1030100001F1080EAFEC07F0E8CF02F1090EAFECBA
:1030200007F0E8CF03F11EEF18F0010183EC1DF06B
:10303000078457C100F158C101F107940101E80E5E
:10304000046F800E056F000E066F000E076F9BEC7D
:103050001CF0000E046F040E056F000E066F000ECC
:10306000076FBAEC1CF0880E046F130E056F000E8C
:10307000066F000E076F8CEC1CF00A0E046F000E3A
:10308000056F000E066F000E076FBAEC1CF026EC01
:103090001DF00101296752EF18F00401200E826F24
:1030A00055EF18F004012D0E826F69EC0AF030C163
:1030B00082F40401300E822769EC0AF031C182F4F7
:1030C0000401300E822769EC0AF032C182F4040157
:1030D000300E822769EC0AF004012E0E826F69EC33
:1030E0000AF033C182F40401300E822769EC0AF041
:1030F0000401430E826F69EC0AF0120087C32AF1C3
:1031000088C32BF189C32CF18AC32DF18BC32EF117
:103110008CC32FF18DC330F18EC331F190C332F1E6
:1031200091C333F10101296BD1EC1DF048EC1DF086
:103130000101000E046F000E056F010E066F000EF8
:10314000076F9BEC1CF00E0E0C6E00C10BF099EC9F
:1031500007F00F0E0C6E01C10BF099EC07F0100E8A
:103160000C6E02C10BF099EC07F0110E0C6E03C14E
:103170000BF099EC07F004017A0E826F69EC0AF00B
:1031800004012C0E826F69EC0AF00401350E826F87
:1031900069EC0AF004012C0E826F69EC0AF0FAEC7B
:1031A00016F002EF13F087C32AF188C32BF189C30D
:1031B0002CF18AC32DF18BC32EF18CC32FF18DC35B
:1031C00030F18EC331F190C332F191C333F101017B
:1031D000296BD1EC1DF048EC1DF0880E046F130E26
:1031E000056F000E066F000E076F90EC1CF0000ECE
:1031F000046F040E056F000E066F000E076F9BEC48
:103200001CF00101E80E046F800E056F000E066FC2
:10321000000E076FBAEC1CF00A0E0C6E00C10BF02A
:1032200099EC07F00B0E0C6E01C10BF099EC07F056
:103230000C0E0C6E02C10BF099EC07F00D0E0C6E2B
:1032400003C10BF099EC07F004017A0E826F69EC70
:103250000AF004012C0E826F69EC0AF00401360EAC
:10326000826F69EC0AF004012C0E826F69EC0AF09F
:10327000E9EC17F002EF13F087C32AF188C32BF1B2
:1032800089C32CF18AC32DF18BC32EF18CC32FF18E
:103290008DC330F18FC331F190C332F191C333F15B
:1032A0000101D1EC1DF048EC1DF0000E046F120E70
:1032B000056F000E066F000E076F9BEC1CF00101FE
:1032C0000A0E046F000E056F000E066F000E076FEA
:1032D000BAEC1CF0120E0C6E00C10BF099EC07F06A
:1032E000130E0C6E01C10BF099EC07F0140E0C6E6E
:1032F00002C10BF099EC07F0150E0C6E03C10BF038
:1033000099EC07F004017A0E826F69EC0AF004016F
:103310002C0E826F69EC0AF00401370E826F69ECA3
:103320000AF004012C0E826F69EC0AF06DEC17F0C4
:1033300002EF13F087C32AF188C32BF189C32CF164
:103340008AC32DF18BC32EF18CC32FF18DC330F1C5
:103350008EC331F190C332F191C333F10101296B76
:10336000D1EC1DF048EC1DF0880E046F130E056FB4
:10337000000E066F000E076F90EC1CF0000E046F3D
:10338000040E056F000E066F000E076F9BEC1CF01D
:103390000101E80E046F800E056F000E066F000E2F
:1033A000076FBAEC1CF0060E0C6E00C10BF099EC26
:1033B00007F0070E0C6E01C10BF099EC07F0080E38
:1033C0000C6E02C10BF099EC07F0090E0C6E03C1F4
:1033D0000BF099EC07F004017A0E826F69EC0AF0A9
:1033E00004012C0E826F69EC0AF00401380E826F22
:1033F00069EC0AF004012C0E826F69EC0AF0FFEC14
:1034000017F002EF13F081A8C1EF1AF007A87AEFC6
:103410001AF00101800E006F1A0E016F060E026F86
:10342000000E036F4BC104F14CC105F14DC106F113
:103430004EC107F18CEC1CF003BFC1EF1AF02BEC6E
:103440001BF04BC100F14CC101F14DC102F14EC165
:1034500003F1078299EC1BF018C104F119C105F1C1
:103460001AC106F11BC107F1F80E006FCD0E016FF6
:10347000660E026F030E036F8CEC1CF00E0E0C6ECA
:1034800000C10BF099EC07F00F0E0C6E01C10BF0B0
:1034900099EC07F0100E0C6E02C10BF099EC07F0DE
:1034A000110E0C6E03C10BF099EC07F007840101BB
:1034B00083EC1DF057C100F158C101F107940A0EC9
:1034C0000C6E00C10BF099EC07F00B0E0C6E01C1F5
:1034D0000BF099EC07F00C0E0C6E02C10BF099EC9E
:1034E00007F00D0E0C6E03C10BF099EC07F0079876
:1034F000C1EF1AF007AAC1EF1AF00784010183ECAB
:103500001DF057C100F158C101F10794060E0C6E71
:1035100000C10BF099EC07F0070E0C6E01C10BF027
:1035200099EC07F0080E0C6E02C10BF099EC07F055
:10353000090E0C6E03C10BF099EC07F0078462C111
:1035400000F163C101F164C102F165C103F10794A7
:10355000120E0C6E00C10BF099EC07F0130E0C6EFE
:1035600001C10BF099EC07F0140E0C6E02C10BF0C8
:1035700099EC07F0150E0C6E03C10BF099EC07F0F7
:10358000079A0401805181197F0B0BE09EA809D096
:1035900014EE00F081517F0BE126E750812B0F01E3
:1035A000AD6E05012951010A13E081AAE8EF1AF076
:1035B00005012951000A0AE00EB8E8EF1AF00501EA
:1035C0002A67E8EF1AF00EB8E8EF1AF0F0EF23F0F0
:1035D00081B8FDEF1AF0CAEC1EF005012951020A6C
:1035E00002E0FDEF1AF0562FFDEF1AF055C556F523
:1035F0000501010E2A6F3C0E2B6FD7EF09F018C1A1
:1036000000F119C101F11AC102F11BC103F1000E51
:10361000046F000E056F010E066F000E076FBAEC07
:103620001CF029A12AEF1BF02051D8B42AEF1BF07F
:1036300018C100F119C101F11AC102F11BC103F156
:10364000000E046F000E056F0A0E066F000E076F66
:10365000BAEC1CF012000101186B196B1A6B1B6B92
:1036600012002AC182F40401300E822769EC0AF0AC
:103670002BC182F40401300E822769EC0AF02CC1C0
:1036800082F40401300E822769EC0AF02DC182F425
:103690000401300E822769EC0AF02EC182F4040185
:1036A000300E822769EC0AF02FC182F40401300E3B
:1036B000822769EC0AF030C182F40401300E8227BF
:1036C00069EC0AF031C182F40401300E822769EC02
:1036D0000AF032C182F40401300E822769EC0AF04C
:1036E00033C182F40401300E822769EC0AF0120023
:1036F000060E106E060E116E060E126E102E7EEF66
:103700001BF0112E7EEF1BF0122E7EEF1BF08B8430
:10371000020E106E020E116E020E126E102E8EEF41
:103720001BF0112E8EEF1BF0122E8EEF1BF08B94E0
:1037300012000101005305E1015303E1025301E1CD
:10374000002B5CEC1CF083EC1DF03951006F3A51FA
:10375000016F420E046F4B0E056F000E066F000ED8
:10376000076F9BEC1CF000C104F101C105F102C11F
:1037700006F103C107F118C100F119C101F11AC125
:1037800002F11BC103F107B2CAEF1BF090EC1CF071
:10379000CCEF1BF08CEC1CF000C118F101C119F149
:1037A00002C11AF103C11BF1120083EC1DF059C1D3
:1037B00000F15AC101F1060EAFEC07F0E8CF04F1B9
:1037C000070EAFEC07F0E8CF05F1080EAFEC07F0FD
:1037D000E8CF06F1090EAFEC07F0E8CF07F18CEC6B
:1037E0001CF000C124F101C125F102C126F103C181
:1037F00027F1290E046F000E056F000E066F000EF4
:10380000076F9BEC1CF0EE0E046F430E056F000E6D
:10381000066F000E076F90EC1CF024C104F125C167
:1038200005F126C106F127C107F19BEC1CF000C190
:103830001CF101C11DF102C11EF103C11FF1120EE5
:10384000AFEC07F0E8CF04F1130EAFEC07F0E8CFD0
:1038500005F1140EAFEC07F0E8CF06F1150EAFEC52
:1038600007F0E8CF07F10D0E006F000E016F000E9C
:10387000026F000E036F9BEC1CF0180E046F000E1D
:10388000056F000E066F000E076FBAEC1CF01CC12E
:1038900004F11DC105F11EC106F11FC107F190EC35
:1038A0001CF06A0E046F2A0E056F000E066F000EE4
:1038B000076F8CEC1CF01200BF0EFA6E200E3A6FF0
:1038C000396BD8900037013702370337D8B06DEF26
:1038D0001CF03A2F62EF1CF039073A070353D8B4B3
:1038E00012000331070B80093F6F03390F0B010FE3
:1038F000396F80EC5FF0406F390580EC5FF0405D20
:10390000405F396B3F33D8B0392739333FA982EF55
:103910001CF0405139271200A8EC1DF0D8B012005D
:1039200003510719346F6BEC1DF0D8900751031940
:1039300034AF800F1200346B8FEC1DF0D8A0A5ECD3
:103940001DF0D8B012007AEC1DF083EC1DF01F0EB4
:10395000366FBBEC1DF00B35D8B06BEC1DF0D8A06A
:103960000335D8B01200362FA9EF1CF034B192EC19
:103970001DF01200346B04510511061107110008E7
:10398000D8A08FEC1DF0D8A0A5EC1DF0D8B0120087
:10399000086B096B0A6B0B6BBBEC1DF01F0E366FCF
:1039A000BBEC1DF007510B5DD8A4E3EF1CF00651F2
:1039B0000A5DD8A4E3EF1CF00551095DD8A4E3EF3C
:1039C0001CF00451085DD8A0F6EF1CF00451085F0C
:1039D0000551D8A0053D095F0651D8A0063D0A5FF4
:1039E0000751D8A0073D0B5FD8900081362FD0EF4C
:1039F0001CF034B192EC1DF0346B8FEC1DF0D890BC
:103A0000BFEC1DF007510B5DD8A413EF1DF006515C
:103A10000A5DD8A413EF1DF00551095DD8A413EF7A
:103A20001DF00451085DD8A022EF1DF0003F22EFE9
:103A30001DF0013F22EF1DF0023F22EF1DF0032B8E
:103A4000D8B4120034B192EC1DF012000101346BB5
:103A50008FEC1DF0D8B01200C4EC1DF0200E366FB4
:103A6000003701370237033711EE33F00A0E376F94
:103A7000E7360A0EE75CD8B0E76EE552372F38EF2D
:103A80001DF0362F30EF1DF034B12981D89012008F
:103A900001010A0E346F200E366F11EE29F03451F9
:103AA000376F0A0ED890E652D8B0E726E732372FA4
:103AB00053EF1DF00333023301330033362F4DEF44
:103AC0001DF0E750FF0FD8A00335D8B0120029B180
:103AD00092EC1DF01200045100270551D8B0053DAD
:103AE00001270651D8B0063D02270751D8B0073D3F
:103AF000032712000051086F0151096F02510A6F2C
:103B000003510B6F12000101006B016B026B036B21
:103B100012000101046B056B066B076B1200033585
:103B2000D8A012000351800B001F011F021F031FAA
:103B3000003FA2EF1DF0013FA2EF1DF0023FA2EFF8
:103B40001DF0032B342B032512000735D8A01200DB
:103B50000751800B041F051F061F071F043FB8EF06
:103B60001DF0053FB8EF1DF0063FB8EF1DF0072B25
:103B7000342B072512000037013702370337083787
:103B800009370A370B3712000101296B2A6B2B6B9F
:103B90002C6B2D6B2E6B2F6B306B316B326B336B51
:103BA00012002A510F0B2A6F2B510F0B2B6F2C5128
:103BB0000F0B2C6F2D510F0B2D6F2E510F0B2E6FE6
:103BC0002F510F0B2F6F30510F0B306F31510F0BE7
:103BD000316F32510F0B326F33510F0B336F1200B5
:103BE0008984000EC76E220EC66E9E96C69E000E7B
:103BF000C96EFF0E9EB602D0E82EFCD79E96C69EDA
:103C0000000EC96EFF0E9EB602D0E82EFCD7C9CFBB
:103C1000A5F59E96C69E000EC96EFF0E9EB602D0FA
:103C2000E82EFCD7C9CFA6F59E96C69E000EC96E9B
:103C3000FF0E9EB602D0E82EFCD7C9CFA7F59E9600
:103C4000C69E000EC96EFF0E9EB602D0E82EFCD7AF
:103C5000C9CFA8F59E96C69E000EC96EFF0E9EB6F1
:103C600002D0E82EFCD7C9CFA9F59E96C69E000EBD
:103C7000C96EFF0E9EB602D0E82EFCD7C9CFAAF5BA
:103C80009E96C69E000EC96EFF0E9EB602D0E82E0E
:103C9000FCD7C9CFABF58994CDEC20F01200898414
:103CA000000EC76E220EC66E9E96C69E800EC96E10
:103CB000FF0E9EB602D0E82EFCD79E96C69EA5C5E6
:103CC000C9FFFF0E9EB602D0E82EFCD79E96C69E78
:103CD000A6C5C9FFFF0E9EB602D0E82EFCD79E9661
:103CE000C69EA7C5C9FFFF0E9EB602D0E82EFCD720
:103CF0009E96C69EA8C5C9FFFF0E9EB602D0E82EAE
:103D0000FCD79E96C69EA9C5C9FFFF0E9EB602D0DF
:103D1000E82EFCD79E96C69EAAC5C9FFFF0E9EB68A
:103D200002D0E82EFCD79E96C69EABC5C9FFFF0EFB
:103D30009EB602D0E82EFCD78994CDEC20F02B0E55
:103D40000C6EA5C50BF099EC07F02C0E0C6EA6C5F9
:103D50000BF099EC07F02D0E0C6EA7C50BF099EC4B
:103D600007F02E0E0C6EA8C50BF099EC07F02F0E85
:103D70000C6EA9C50BF099EC07F0300E0C6EAAC5BD
:103D80000BF099EC07F0310E0C6EABC50BF099EC13
:103D900007F012008984000EC76E220EC66E9E9632
:103DA000C69E070EC96EFF0E9EB602D0E82EFCD747
:103DB0009E96C69E000EC96EFF0E9EB602D0E82EDD
:103DC000FCD7C9CFA5F59E96C69E000EC96EFF0E04
:103DD0009EB602D0E82EFCD7C9CFA6F59E96C69E09
:103DE000000EC96EFF0E9EB602D0E82EFCD7C9CFDA
:103DF000A7F59E96C69E000EC96EFF0E9EB602D017
:103E0000E82EFCD7C9CFA8F58994CDEC20F08984A1
:103E1000000EC76E220EC66E9E96C69E0F0EC96E0F
:103E2000FF0E9EB602D0E82EFCD79E96C69E000ED0
:103E3000C96EFF0E9EB602D0E82EFCD7C9CFADF5F5
:103E40008994CDEC20F012008984000EC76E220EFA
:103E5000C66E9E96C69E870EC96EFF0E9EB602D097
:103E6000E82EFCD79E96C69EA5C5C9FFFF0E9EB63E
:103E700002D0E82EFCD79E96C69EA6C5C9FFFF0EAF
:103E80009EB602D0E82EFCD79E96C69EA7C5C9FF57
:103E9000FF0E9EB602D0E82EFCD79E96C69EA8C501
:103EA000C9FFFF0E9EB602D0E82EFCD78994CDEC58
:103EB00020F089849E96C69E8F0EC96EFF0E9EB618
:103EC00002D0E82EFCD79E96C69EADC5C9FFFF0E58
:103ED0009EB602D0E82EFCD78994CDEC20F01200DB
:103EE0008984000EC76E220EC66E9E96C69E870EF1
:103EF000C96EFF0E9EB602D0E82EFCD79E96C69ED7
:103F0000000EC96EFF0E9EB602D0E82EFCD79E961C
:103F1000C69E800EC96EFF0E9EB602D0E82EFCD75C
:103F20009E96C69E800EC96EFF0E9EB602D0E82EEB
:103F3000FCD79E96C69E800EC96EFF0E9EB602D01E
:103F4000E82EFCD78994CDEC20F089849E96C69EFD
:103F50008F0EC96EFF0E9EB602D0E82EFCD79E963D
:103F6000C69E010EC96EFF0E9EB602D0E82EFCD78B
:103F70008994CDEC20F012008984000EC76E220EC9
:103F8000C66E9E96C69E870EC96EFF0E9EB602D066
:103F9000E82EFCD79E96C69E000EC96EFF0E9EB6FA
:103FA00002D0E82EFCD79E96C69E000EC96EFF0E6C
:103FB0009EB602D0E82EFCD79E96C69E800EC96E95
:103FC000FF0E9EB602D0E82EFCD79E96C69E800EAF
:103FD000C96EFF0E9EB602D0E82EFCD78994CDECB8
:103FE00020F089849E96C69E8F0EC96EFF0E9EB6E7
:103FF00002D0E82EFCD79E96C69E010EC96EFF0E1B
:104000009EB602D0E82EFCD78994CDEC20F01200A9
:104010008984000EC76E220EC66E9E96C69E8F0EB7
:10402000C96EFF0E9EB602D0E82EFCD7CDEC20F074
:104030009E96C69E810EC96EFF0E9EB602D0E82ED9
:10404000FCD78994CDEC20F08984000EC76E220E37
:10405000C66E9E96C69E8F0EC96EFF0E9EB602D08D
:10406000E82EFCD7CDEC20F09E96C69E010EC96EC0
:10407000FF0E9EB602D0E82EFCD78994CDEC20F03E
:1040800089849E96C69E910EC96EFF0E9EB602D082
:10409000E82EFCD7CDEC20F09E96C69EA50EC96EEC
:1040A000FF0E9EB602D0E82EFCD78994CDEC20F00E
:1040B00012008984000EC76E220EC66E9E96C69EA2
:1040C0008F0EC96EFF0E9EB602D0E82EFCD7CDEC47
:1040D00020F09E96C69E810EC96EFF0E9EB602D03F
:1040E000E82EFCD78994CDEC20F012008984000ED4
:1040F000C76E220EC66E9E96C69E8F0EC96EFF0EAE
:104100009EB602D0E82EFCD7CDEC20F09E96C69E3F
:10411000010EC96EFF0E9EB602D0E82EFCD7899420
:10412000CDEC20F012008984000EC76E220EC66E00
:104130009E96C69E910EC96EFF0E9EB602D0E82EC8
:10414000FCD7CDEC20F09E96C69EA50EC96EFF0E44
:104150009EB602D0E82EFCD78994CDEC20F0120058
:104160008984000EC76E220EC66E9E96C69E910E64
:10417000C96EFF0E9EB602D0E82EFCD7CDEC20F023
:104180009E96C69E000EC96EFF0E9EB602D0E82E09
:10419000FCD78994CDEC20F01200050EE82EFED756
:1041A0001200200EC66E0501256B266B276B286B4F
:1041B000899A400EC76E200EC66E9E96C69E030E4E
:1041C000C96EFF0E9EB602D0E82EFCD79E96C69E04
:1041D00027C5C9FFFF0E9EB602D0E82EFCD79E96DB
:1041E000C69E26C5C9FFFF0E9EB602D0E82EFCD79C
:1041F0009E96C69E25C5C9FFFF0E9EB602D0E82E2C
:10420000FCD79E96C69EC952FF0E9EB602D0E82EDF
:10421000FCD7898AC950FF0A02E118EF21F0100E7D
:104220002527E86A2623E86A272327A9D8EF20F064
:10423000220EC66E1200899A400EC76E200EC66E00
:104240009E96C69E060EC96EFF0E9EB602D0E82E42
:10425000FCD7898A899A9E96C69EC70EC96EFF0EA4
:104260009EB602D0E82EFCD7898A899A9E96C69E71
:10427000050EC96EFF0E9EB602D0E82EFCD79E96A4
:10428000C69EC952FF0E9EB602D0E82EFCD7C9B01A
:104290003FEF21F0898A0501256B266B276B286B80
:1042A00012000501FE0E2D6F0501000E2D6FF0ECC2
:1042B0001DF0A5C52EF5A6C52FF5A7C530F5A8C5D7
:1042C00031F5A9C532F5AAC533F5ABC534F5078478
:1042D000B6C166F1B7C167F1B8C168F1B9C169F19A
:1042E0004BC14FF14CC150F14DC151F14EC152F192
:1042F00057C159F158C15AF107942CEC13F000C181
:1043000035F501C136F502C137F503C138F50501B0
:10431000576792EF21F0586792EF21F0596792EFBB
:1043200021F05A6796EF21F0A4EF21F057C504F170
:1043300058C505F159C506F15AC507F101018CECC4
:104340001CF003BF12EF22F059C139F55AC13AF5FA
:10435000AFC53BF5B0C53CF50501100E2C6F899A31
:10436000400EC76E200EC66E9E96C69E060EC96E85
:10437000FF0E9EB602D0E82EFCD7898A899A9E96B7
:10438000C69E020EC96EFF0E9EB602D0E82EFCD766
:104390009E96C69E27C5C9FFFF0E9EB602D0E82E88
:1043A000FCD79E96C69E26C5C9FFFF0E9EB602D0BC
:1043B000E82EFCD79E96C69E25C5C9FFFF0E9EB669
:1043C00002D0E82EFCD725EE2DF02C2F02D0F4EFF2
:1043D00021F09E96C69EDECFC9FFFF0E9EB602D08C
:1043E000E82EFCD7E5EF21F0898A899A9E96C69E31
:1043F000050EC96EFF0E9EB602D0E82EFCD79E9623
:10440000C69EC952FF0E9EB602D0E82EFCD7C9B098
:10441000FFEF21F0898A0501100E2527E86A26237F
:10442000E86A2723120019C502F51AC503F525EE1F
:104430005FF005012C6B16EE00F005010251E1263C
:104440000351D8B00329E226E7CFE8FF2C0A06E1A2
:104450002CC5DEFF05012C6B36EF22F0E7CFE8FF1D
:104460002A0A0CE0E7CFDEFF05012C2B0501032B08
:10447000023F0307030E03171BEF22F005012D6B0C
:104480002E6B2F6B306B316B326B336B346B356B48
:10449000366B376B386B396B3A6B3B6B3C6B3D6BF8
:1044A0003E6B3F6B406B416B426B436B446B456BA8
:1044B000466B476B486B496B4A6B4B6B4C6BDDCF64
:1044C000E8FF05012C5105E0DDCFE8FF2C2F64EF5C
:1044D00022F00501DDCF2CF52C5105E0DDCFE8FF02
:1044E0002C2F6EEF22F00501DDCF2CF52C5105E0CD
:1044F000DDCFE8FF2C2F78EF22F011EE33F0010131
:10450000C4EC1DF00501DDCF2CF52C5105E0DDCF0D
:10451000E5FF2C2F87EF22F00101D1EC1DF048ECD4
:104520001DF000C12EF501C12FF502C130F50501C6
:10453000DDCF2CF52C5105E0DDCFE8FF2C2F9CEFD3
:1045400022F00501DDCF2CF52C5105E0DDCFE8FF91
:104550002C2FA6EF22F00501DDCF2CF52C5107E022
:10456000DDCFE8FFE8A82D852C2FB0EF22F011EE6B
:1045700033F00101C4EC1DF00501DDCF2CF52C5109
:1045800014E0DDCFE5FFDDCFE5FFDDCFE5FFDDCFDB
:10459000E5FFDDCFE8FFDDCFE5FFDDCFE5FFDDCFD8
:1045A000E5FFDDCFE5FFDDCFE5FF0101D1EC1DF03B
:1045B00048EC1DF000C138F501C139F502C13AF5EA
:1045C00003C13BF50501DDCF2CF52C5107E0DDCF14
:1045D000E8FFE8A82D832C2FE7EF22F011EE33F04F
:1045E0000101C4EC1DF00501DDCF2CF52C5105E0D7
:1045F000DDCFE5FF2C2FF8EF22F001012EC12FF1C6
:104600002DC12EF12CC12DF12BC12CF1D1EC1DF0BF
:1046100048EC1DF000C134F501C135F502C136F595
:1046200003C137F50501DDCF2CF52C5107E0DDCFB7
:10463000E8FF2C2F17EF23F0E8B02D8711EE33F0B1
:104640000101C4EC1DF0DDCFE8FFDDCFE8FFDDCFD9
:10465000E8FFDDCFE8FFDDCFE8FFDDCFE5FFDDCF11
:10466000E5FFDDCFE5FFDDCFE5FFDDCFE5FFDDCF0A
:10467000E5FFD1EC1DF048EC1DF000C131F501C1A2
:1046800032F502C133F5078462C166F163C167F197
:1046900064C168F165C169F14BC14FF14CC150F182
:1046A0004DC151F14EC152F157C159F158C15AF1A2
:1046B00007942CEC13F000C13CF501C13DF502C19B
:1046C0003EF503C13FF5120021C500F122C501F1FD
:1046D00023C502F124C503F1899A400EC76E200E4E
:1046E000C66E9E96C69E0B0EC96EFF0E9EB602D07B
:1046F000E82EFCD79E96C69E02C1C9FFFF0E9EB64D
:1047000002D0E82EFCD79E96C69E01C1C9FFFF0EBF
:104710009EB602D0E82EFCD79E96C69E00C1C9FF69
:10472000FF0E9EB602D0E82EFCD79E96C69EC952BA
:10473000FF0E9EB602D0E82EFCD725EE2DF0050127
:10474000100E2C6F9E96C69EC952FF0E9EB602D0CA
:10475000E82EFCD7C9CFDEFF2C2FA2EF23F0898AE9
:104760001200899A400EC76E200EC66E9E96C69E97
:10477000900EC96EFF0E9EB602D0E82EFCD79E9614
:10478000C69E000EC96EFF0E9EB602D0E82EFCD764
:104790009E96C69E000EC96EFF0E9EB602D0E82EF3
:1047A000FCD79E96C69E000EC96EFF0E9EB602D026
:1047B000E82EFCD79E96C69EC952FF0E9EB602D02A
:1047C000E82EFCD7C9CF2DF59E96C69EC952FF0E86
:1047D0009EB602D0E82EFCD7C9CF2EF5898A1200EA
:1047E00078EC1BF0AFC5E8FFD70802E378EC1BF0CC
:1047F000AFC5E8FFC80802E378EC1BF0AFC5E8FFDF
:10480000B90802E378EC1BF0AFC5E8FFAA0802E3A1
:1048100078EC1BF0AFC5E8FF9B0802E378EC1BF0D7
:10482000CAEC1EF0F29CF29E8B948A86899CC69AF2
:10483000C2908A94898A9482948C720ED36ED3A487
:10484000FED789968A909390FF0EE8CF00F0E82E6D
:10485000FED7002EFCD78150F294F29A9E909D9044
:104860009E929D92F298F292F290F286F28E03005E
:02487000FF0047
:10BF0000E844F926000C160C2B0C3F0C520C640C68
:10BF1000760C860C960CA50CB30CC10CCF0CDC0C6B
:06BF2000E80CF40C000C1B
:00000001FF
